:10000000800B00206D110000833B0000591100009F
:1000100059110000591100005911000000000000A2
:10002000000000000000000000000000AD0F000014
:100030005911000000000000590F0000013F0000AE
:10004000110F0000110F0000110F0000110F000030
:10005000110F0000110F0000110F0000110F000020
:10006000110F0000110F0000110F0000110F000010
:10007000110F0000110F0000110F0000110F000000
:10008000110F0000110F0000110F0000110F0000F0
:10009000110F0000110F0000110F0000110F0000E0
:1000A000110F0000110F0000110F0000110F0000D0
:1000B000110F0000110F0000110F0000110F0000C0
:1000C000110F0000110F0000110F0000110F0000B0
:0C00D000110F0000110F0000110F0000C4
:1000DC0053B94AB9002908BF00281CBF4FF0FF31A3
:1000EC004FF0FF3000F06CB9ADF1080C6DE904CEA7
:1000FC0000F006F8DDF804E0DDE9022304B07047F7
:10010C002DE9F047089E0D4604468E46002B40F024
:10011C0082808A42174646D9B2FA82F24AB1C2F1BB
:10012C00200105FA02F320FA01F1974041EA030E8F
:10013C0094404FEA1748230CBEFBF8FCB9B208FBFD
:10014C001CEE43EA0E430CFB01F098420AD9FB1853
:10015C000CF1FF3580F01681984240F21381ACF11E
:10016C00020C3B441B1AA4B2B3FBF8F008FB10338F
:10017C0044EA034400FB01F1A14209D93C1900F106
:10018C00FF3380F00181A14240F2FE8002383C44F2
:10019C00641A40EA0C4000211EB1D4400023C6E989
:1001AC000043BDE8F08702B9FFDEB2FA82F2002A02
:1001BC004FD1CB1B4FEA174E1FFA87F80121B3FB27
:1001CC00FEFC250C0EFB1C3345EA034508FB0CF327
:1001DC00AB4207D97D190CF1FF3002D2AB4200F2D1
:1001EC00E7808446ED1AA3B2B5FBFEF00EFB10556A
:1001FC0043EA054408FB00F8A04507D93C1900F177
:10020C00FF3302D2A04500F2D7801846A4EB0804B5
:10021C0040EA0C40C0E78B4208D9002E00F0AF80BA
:10022C000021C6E900050846BDE8F087B3FA83F162
:10023C0000294BD1AB4202D3824200F2B780841A20
:10024C0065EB030301209E46002EAAD0C6E9004EA2
:10025C00A7E7C2F1200C01FA02F3974020FA0CF048
:10026C004FEA174E21FA0CFC1843BCFBFEF1050CAF
:10027C000EFB11CC1FFA87F845EA0C4501FB08F37D
:10028C00AB4204FA02F409D97D1901F1FF3C80F06C
:10029C008B80AB4240F2888002393D44EB1A85B228
:1002AC00B3FBFEF00EFB103345EA034500FB08F3ED
:1002BC00AB4207D97D1900F1FF3C71D2AB426FD92B
:1002CC0002383D44EB1A40EA014178E7C1F1200CB9
:1002DC008B4022FA0CF71F4320FA0CF405FA01F3B9
:1002EC004FEA174E25FA0CF51C43230CB5FBFEF90F
:1002FC001FFA87F80EFB195543EA054509FB08FA66
:10030C00AA4502FA01F200FA01F308D97D1909F1A4
:10031C00FF3047D2AA4545D9A9F102093D44A5EBC6
:10032C000A05A4B2B5FBFEF00EFB105544EA0544D9
:10033C0000FB08F8A04507D93C1900F1FF352DD278
:10034C00A0452BD902383C4440EA0940A4EB0804F0
:10035C00A0FB02894C45C6464D4619D316D05EB15A
:10036C00B3EB0E0264EB050404FA0CFCCA404CEA35
:10037C000202CC40C6E900240021BDE8F0873146DA
:10038C0030460EE7AC46EDE6184601E74345E6D2AB
:10039C00B8EB020E69EB07050138E0E72846D3E716
:1003AC0060468FE78146BAE7614677E708464BE738
:1003BC00ACF1020C3D4415E702383C4426E700BF83
:1003CC00704700BF70B5164802F010FC044630B3FD
:1003DC0002698168136843F4003313600B6840F2C0
:1003EC00016211219847002819DB012523691B683C
:1003FC0085F0010613F4003F18BFF5B265B1A36890
:10040C00DB684FF4003120469847F5B200214FF4D9
:10041C00004002F08DFFE9E7A3681B69F1E770BDAE
:10042C005C4400002DE9F04F91B08B46029092464F
:10043C001C4600259AF8000008B928465EE32528DA
:10044C000AF1010707D0029B594698470028C0F2D1
:10045C005583013510E2182200210AA803F0C6FBCF
:10046C009AF80130252B78D00022944616469646F1
:10047C001046394617F8013B2B2B00F09D8000F2FB
:10048C009480202B00F09B80232B00F09A8028B1C5
:10049C009DF8300040F004008DF83000BEF1000FE4
:1004AC0005D09DF8300040F008008DF830002EB1DA
:1004BC009DF8300040F010008DF83000BCF1000FBA
:1004CC0005D09DF8300040F020008DF830002AB1A6
:1004DC009DF8302042F040028DF830209DF83020FD
:1004EC0002F04400442803D16FF386128DF83020BB
:1004FC009DF830202A2B42F080028DF830207BD1E1
:10050C009DF8312042F001024B1C8DF831201A78F5
:10051C002E2A9DF831200CBF0121002161F34102EC
:10052C008DF8312074D15A782A2A6AD001330021EF
:10053C000A26184610F8012BA2F13007092F40F2B9
:10054C008E809DF830200E91C2F3400040EAD171AC
:10055C0061F341028DF830205AE00AF102078DF860
:10056C0033309DF83130D90740F1498154F8049B60
:10057C00B9F1000F07DA9DF8302042F004028DF833
:10058C003020C9F100095A0740F1428154F8048B1C
:10059C00B8F1000F80F241819DF831306FF34103C7
:1005AC008DF831304FF0FF3837E12D2B0CD0302B3C
:1005BC007FF46DAF01225CE74FF0010E59E7012685
:1005CC0057E74FF0010C54E7012052E70CFB0202F5
:1005DC00303A33461E4616F8010BA0F13007092FAE
:1005EC00F4D9994293D09DF830100D92D20F62F34A
:1005FC0041018DF830108AE70B4600224FF00A0CAF
:10060C00E8E79DF8312042F004028DF831200233E6
:10061C001F4617F8012B6C2A41D025D8682A2BD0FD
:10062C006A2A46D04C2A4CD01F4617F8012B9DF84D
:10063C0031308DF83320782A00F2D980572A4DD8E2
:10064C00412A03D0453A022A00F2D1809DF832307B
:10065C00042262F302038DF8323001239EE006FB84
:10066C0001213039034664E7742A26D07A2ADBD17B
:10067C009DF8313006220DE05A78682A9DF8312019
:10068C0006D1012161F3C6028DF831209F1CCCE705
:10069C001346022262F3C6038DF83130C5E75A784F
:1006AC006C2A9DF8312001D10421EBE7134603227B
:1006BC00F0E79DF831300522ECE79DF83130072248
:1006CC00E8E7BDF8303023F4F04323F0020343F4A1
:1006DC00804343F00203ADF83030A6E7A2F1580195
:1006EC00202900F2848001A050F821F0BD07000001
:1006FC00FB070000FB070000FB070000FB070000E6
:10070C00FB070000FB070000FB070000FB070000D5
:10071C0059060000FB070000BD0700007D07000024
:10072C00590600005906000059060000FB0700009E
:10073C007D070000FB070000FB070000FB07000023
:10074C00FB070000C5070000BD070000E107000023
:10075C00FB070000FB070000E1070000FB0700009F
:10076C00BD070000FB070000FB070000BD070000F1
:10077C009DF83210012003F0780360F30201402B46
:10078C008DF8321002BF9DF8301041F001018DF848
:10079C003010632A31D1003B18BF01239DF8302063
:1007AC00C2F340010B4363F341028DF83020D8E6CD
:1007BC009DF832100220DEE79DF8322003F078031A
:1007CC00A3F14000032161F3020243428DF8322071
:1007DC004341E3E79DF83220032113F0780F61F3D6
:1007EC0002028DF8322014BF01230023D6E79DF8B6
:1007FC00303043F001038DF830300023CEE79DF903
:10080C003020002AB4BFDDF834904FF0FF39BAE63F
:10081C009B077FF5C7AEDDF838809DF831200023AB
:10082C00CDE90D339DF8323003F00703012BC2F3F1
:10083C00C30236D1D31E042B20D8DFE803F0030704
:10084C00071F1F0054F8040BC11704E0073424F0F1
:10085C000704F4E80201CDE90A019DF8303013F0E9
:10086C00030654D002983B465246594603F07BF897
:10087C000028C0F243810544BA46DBE554F8040B6A
:10088C00012A4FEAE071CDE90A0105D19DF8283023
:10089C000A9300230B93E0E7022ADED1BDF928006E
:1008AC00D2E7022B23D1D31E042B13D8DFE803F09D
:1008BC00030A0A12120020680A900021231D0B91D2
:1008CC001C46CAE7073424F00703F3E80201CDE91C
:1008DC000A01F5E754F8043B0A93012A4FF0000390
:1008EC000B93D3D0022AB8D1BDF82830D0E7042B13
:1008FC0007D1073424F00704F4E80201CDE90A011A
:10090C00ABE7032B04BF54F8043B0A93A5E79DF80F
:10091C0033007828B0D8622822D825283FF493AD2C
:10092C005828A9D10DF126030093DDE90A0104AB87
:10093C000CAA02F0CDFF8246B8F1000F0DF1260093
:10094C000CDB9DF83020A0EB0A036FF38612984560
:10095C008DF8302002D9A8EB03030D9380463DE0BF
:10096C006338152888D801A151F820F0F909000046
:10097C005D0A00008508000085080000850800005D
:10098C00850800005D0A000085080000850800004D
:10099C008508000085080000BB0A0000890A0000D9
:1009AC008D0A00008508000085080000D1090000B0
:1009BC0085080000890A00008508000085080000F1
:1009CC00890A0000B8F1000FDDF828A00ADB4146C7
:1009DC00504603F0EBF80AEB00080026BAF1000FC2
:1009EC000CD149E7504603F0DAF8F4E70A9B8DF88E
:1009FC00103000260DF111080DF1100AA8EB0A03B6
:100A0C0006B101339DF83220D0066BD50233520665
:100A1C000D9948BF0E9A0B4448BF9B18B9F1000FB3
:100A2C0079DD9DF83020A9EB0309C2F38003039311
:100A3C00530770D4500664D546B1029B59463046D4
:100A4C00984700285ADB039B01351E46302359E09A
:100A5C001E0711D413F0100618BF2026DDE90A2357
:100A6C00002A73F10001BFF65DAF524263EB430302
:100A7C00CDE90A232D2655E72B26EFE7002651E773
:100A8C000A9848B30DF1260300930CAA04AB00217D
:100A9C0002F01EFFBDF8323003F0EF0343F4F043D5
:100AAC0043F010038246ADF83230002644E70A9B2F
:100ABC00072A3FF6E1AEDFE802F00D04060D080848
:100ACC000D0D1D70D8E61D80D6E62846E917C3E942
:100ADC000001D1E61D60CFE6DFF8C4800646A8F120
:100AEC00050A8BE7110748BF013390E718460393BB
:100AFC005946029B98470028039B04DA11B0BDE8C5
:100B0C00F08F20234D444A46002AA5EB090109F138
:100B1C00FF39EBDC0D4636B1029B594630469847FF
:100B2C000028EBDB01359DF83230D90601D41A07C9
:100B3C0006D5029B5946302098470028DEDB01354C
:100B4C009DF83230DB0607D59DF83300029B5946E1
:100B5C0098470028D2DB01350D9E2E44731B002BC9
:100B6C0016DC029843465246594602F0FCFE002819
:100B7C00C4DB0544A944A9EB0503002B7FF77CAE2D
:100B8C00029B5946202098470028B7DB0135F2E735
:100B9C00029B5946302098470028AFDB0135DDE732
:100BAC00684400002DE9F84FB0F8189019F00808C7
:100BBC00044693460DD001290CBF49F0100949F0A9
:100BCC002009A0F818908BF31188BFF36F8FBDE844
:100BDC00F88F09F00709022907D1204602F0F8FE28
:100BEC000028F0D00128238B50D16769218B002F6E
:100BFC0015DA256821F00701C4E9008841F00101EC
:100C0C0021830026218B01F0070ACA4502D0A36874
:100C1C00002B5CD10DB9002E74D0002358E001F0EC
:100C2C0007035A1F012A20D821F00701062B25683B
:100C3C0089B2C4E900880CD1002D2B4638BF0023A3
:100C4C002BB1628B1B6801326283002BF8D141F00F
:100C5C0002012183204602F0BBFE06460028D1D0BB
:100C6C00238B43F020032383CBE7042B0CD121F0FF
:100C7C00070189B22183204602F0AAFE054600280E
:100C8C00BFD041F0200121830025BAE7032809D108
:100C9C00226923F00703166843F00603238300251B
:100CAC002F46AFE7042806D1226923F007035668C4
:100CBC0043F00403F2E7052806D1226923F0070369
:100CCC00966843F00503E9E700252E46E8E7012383
:100CDC0041F0080121838BF31188BFF36F8F03BBA5
:100CEC00002D33D116B121492046B0474FF02003D7
:100CFC00EFF3118B83F31288BFF36F8F238B23F0E9
:100D0C0008032383238BDA0628D523F010032383CF
:100D1C000121B4F8189009F0070900297FF45BAFA2
:100D2C0051E7A1680029DBD00B68D1F804B0002B87
:100D3C0038BF0023994652463B462046D847B9F166
:100D4C00000FCDD0D9F800304946EEE729463B4696
:100D5C00524620462D6802F057FEC1E713F02001E1
:100D6C001EBF23F0200323830221D2E7413A000067
:100D7C00F8B505464FF02003EFF3118683F3128884
:100D8C00BFF36F8F0B4B1C68002C38BF00245CB179
:100D9C00094FD4E90132002D08BF13460BB1387846
:100DAC0098472468002CF4D186F31188BFF36F8F19
:100DBC00F8BD00BF68010020700100201FB50F4B6B
:100DCC001A68BAB901221A600D4A07CA01AB83E846
:100DDC0007000C4A4AB193E8070002F023FF0020F9
:100DEC0005B05DF804EBFFF7C3BF82F31188BFF3C6
:100DFC006F8FF4E705B05DF804FB00BF0000002026
:100E0C0070010020313C0000F0B589B06E460146FF
:100E1C000546304602F087FE96E80700174C84E83A
:100E2C000700207840B3164B002119606B1C0ED0C4
:100E3C00144817464FF400460021134A0023E6FBE2
:100E4C000701FFF745F90121281A03F06FF902F0A9
:100E5C002BF80120FFF78CFF94E8070005AB83E823
:100E6C0007000A4A1AB193E8070002F0C8FEFFF720
:100E7C00A5FF02F0A7F9207809B0F0BD70010020A1
:100E8C00000000203F420F0040420F000B3C0000CE
:100E9C000B6801330B60014B1B68184704000020E2
:100EAC00014B1860704700BF0400002007B50B46CB
:100EBC00002102460191034801A9FFF7B3FA03B0E0
:100ECC005DF804FB9D0E0000014910220A6070477A
:100EDC0010ED00E072B6404080F31188BFF36F8FC5
:100EEC00BFF34F8F30BF62B6BFF36F8F704700BF39
:100EFC0072B6494081F3118820BF80F3118862B625
:100F0C00704700BF01B572B60B4A906900281EBF2E
:100F1C000021916103F02EF862B6EFF30580A0F189
:100F2C0010004FEAC0000549014409C99847BDE8C3
:100F3C000140034908470000200300202442000020
:100F4C003D11000030BFFFF7FDBF00BF12498A689A
:100F5C004FF030001044EFF3098C80E8F01F202094
:100F6C0080F31288BFF36F8F0C4F4FF00066CA6985
:100F7C008A603E60506F0023536780F3118804B57C
:100F8C00104600F075FABDE8044002F1300090E81C
:100F9C00F01F8CF3098870472003002004ED00E05B
:100FAC001EF0040F0CBFEFF30880EFF3098081698A
:100FBC0011F8021C0229FFD001B502F0D4FD01BDCD
:100FCC0043B2002B08DB012200F01F0002FA00F0F4
:100FDC005B09024A42F82300704700BF00E100E0C1
:100FEC00054B420900F01F0053F82220012303FA9D
:100FFC0000F01040704700BF00E100E043B2002B4E
:10100C00A8BF03F1604301F10101B8BF064B4FEAE1
:10101C004111ACBF03F5614300F00F00C9B2B4BF7E
:10102C00195483F80013704714ED00E00B4A08B50F
:10103C000B4B22F07F029A60BFF34F8FBFF36F8F81
:10104C00D3F8882022F47002C3F8882001F056FEF1
:10105C0002F018FC00F0A0F901F05AFE00000000AC
:10106C0000ED00E0094A0A49936809689967094943
:10107C0058674B6843F080534B60002383F311880F
:10108C00BFF36F8F9368986F704700BF20030020E9
:10109C005844000000ED00E042F8203C009B42F870
:1010AC001C3C0A49019B42F8183C029B42F8143C38
:1010BC0021F001014FF0807342F8043C42F8081C07
:1010CC000023203A02654367704700BF5B3B00007A
:1010DC000B4A0346906890B113F1160F406E05D081
:1010EC00A0F120029A4206D8834204D281422CBF3E
:1010FC000021012100E00021002908BF00207047D9
:10110C002003002008B5094B98600D46144600F0EA
:10111C00AFF9204685F30988002163B681F3118865
:10112C00BFF36F8F0022002302F011FD200300207B
:10113C00044B9968D869884203D003494FF0805218
:10114C000A6070472003002004ED00E0EFF30880F4
:10115C00EFF3098101B5724600F092F801BD00BFB2
:10116C00002080F31488BFF36F8F03F003F8002086
:10117C000D490860BFF34F8F0C4880F3088800F0CE
:10118C0027F9202080F3118809484FF40261401898
:10119C0080F30988EFF314800221084380F314884C
:1011AC00BFF36F8FFFF742FF94ED00E0800B002040
:1011BC00000D002038B5194B14469A6A9A6A9A6A3F
:1011CC000546900719D5586B9A6A120615D519B1B0
:1011DC009A6A22F080029A629A6A9A6A9A6AD1068C
:1011EC000ED49B6A9A070BD400200C4A936A43F0E6
:1011FC00FF0393620023237038BD6FF01500EBE7FB
:10120C00064B5B681B05EFD52946FFF761FF0028ED
:10121C00EAD080F309880220E7E700BF00ED00E088
:10122C000D4B9A6A9A6A9A6A920508D59A6B9A6AD1
:10123C00120404D518B19A6A22F400429A62064B41
:10124C009A6A9A6AD20558BF9A6A9A6A002042F43E
:10125C007F429A620870704700ED00E0074B9A6A73
:10126C009A6A9A6A9A6A9A6A9A6A9A6A6FEA0242BD
:10127C006FEA12429A620020704700BF00ED00E056
:10128C0070B53E4B5B688AB00D46C3F3080300266D
:10129C0086F31188BFF36F8F02F07F41B1F17F4F5E
:1012AC0011D102F00C0108290DD0120701D405460A
:1012BC0001260022033B8DF80720032B57D8DFE8CB
:1012CC0003F0044E524B3546F3E72C4BDC6A14F01A
:1012DC0002044CD1DA6A002A18DBDB6A5B0015D5F4
:1012EC00AB6933F8022C4DF602739A420DD003F120
:1012FC00604303F626631B7803B30DF1070201214B
:10130C002846FFF757FF044600E02C689DF807308D
:10131C0093B92022294602A802F05DFC099B46B332
:10132C00C3F3080222B96FEA53236FEA43230993EC
:10133C0002A9204602F015FC0AB070BD104B1B78B8
:10134C002BB10DF107010120FFF76AFFDBE70D4B15
:10135C001B889BB2002BD9D0FFF780FFD3E70DF190
:10136C0007020021CCE70DF107010020ECE7002477
:10137C00CCE723F4FF7323F00103D8E700ED00E082
:10138C0029ED00E02AED00E0024A536943F0100316
:10139C005361704700ED00E0044800232021C2187F
:1013AC000133272B82F80013F9D1704700E100E0DC
:1013BC00064A11680023C1F3072118468B4200D15D
:1013CC007047936010610133F8E700BF90ED00E0C7
:1013DC0008B572B6002383F31388FFF7E9FF144BAB
:1013EC004FF0FF32C3F88020C3F88420C3F8882064
:1013FC00C3F88C20C3F89020C3F89420C3F898202D
:10140C00C3F89C20C3F88021C3F88421C3F8882139
:10141C00C3F88C21C3F89021C3F89421C3F8982108
:10142C00C3F89C2162B6BFF34F8FBFF36F8F08BD1B
:10143C0000E100E0064B9B68834207D1EFF3058384
:10144C0023B1044A536843F08053536001F090BFBA
:10145C002003002000ED00E0024B034A0348012169
:10146C0000F068B800000120000000208843000054
:10147C00426E054B203A1A60044A2021C3E901123E
:10148C001846012100F060B87C01002000000B150B
:10149C00F0B51E4F00268E4201DB1046F0BD4468AD
:1014AC0084B353B104F1FF3C14EA0C0F18D11F2C78
:1014BC0016D905681CEA050F12D1202C0568D0F846
:1014CC0008C0D2B20FD9B4F1004F0ED8013CB4FA17
:1014DC0084F4C4F11F046400072A4CEA040406D9FE
:1014EC006FF01502D9E70824F6E73E24F4E725F05F
:1014FC001F05154345F0100544F00104BA60FD606A
:10150C0001323C6101360C30C5E700BF90ED00E0C4
:10151C00034B05225A60BFF34F8FBFF36F8F704799
:10152C0090ED00E0BFF35F8F014B00225A607047D3
:10153C0090ED00E010B5034C01232278FFF7A8FFD3
:10154C00207010BD5803002008B5084A00231278FB
:10155C00FFF79EFF10F1160F03D0054B0022072852
:10156C0000DD08BD98601A610130F8E758030020CF
:10157C0090ED00E013490868082810B51ED8FFF755
:10158C00D1FF114C49680022904201F10C0105D1A8
:10159C000E4B1870FFF7BCFF002010BDA26051F875
:1015AC000C3C23F01F03134343F01003E36051F88A
:1015BC00043C43F0010323610132E5E74FF0FF30B7
:1015CC00EBE700BF9443000090ED00E058030020CF
:1015DC00014B1860704700BF080000204FF020033B
:1015EC00EFF3118283F31288BFF36F8F0649012347
:1015FC00C1F840354FF08041C1F8783582F311883D
:10160C00BFF36F8F0020704700E001404FF0804324
:10161C00C0B2C3F81C05BFF34F8F0549054BCA6810
:10162C0002F4E0621343CB60BFF34F8F00BFFDE7C2
:10163C0000ED00E00400FA0520B1034B800143F0FB
:10164C0001031847704700BF804300000E4A70B575
:10165C00841AA3100D4C5C430546E4B20C2000FB2D
:10166C0004200E464021084402F0F0FA011E05DB6E
:10167C00074B03EBC40463689847002128463346A4
:10168C00BDE87040184700BF98010020B76DDBB66D
:10169C00C84300002DE9F041104E841BA310104CE0
:1016AC005C43E4B20C256543804605F140000F46CF
:1016BC003044402102F0E3FA011E09DB094A731998
:1016CC00C3E90E27084B53F83430BDE8F0411847F6
:1016DC0040463B46BDE8F041184700BF980100204A
:1016EC00B76DDBB6ED3C0000C8430000002270B5BE
:1016FC00012104461046FFF781FC0020FFF760FC37
:10170C000F4800F055FF0F4B984215D102F0F8FB33
:10171C0026690D49304602F0AAF900280BDB012599
:10172C0035642469084904F11C0002F0A0F9002872
:10173C0001DBE564002070BD6FF00400FBE700BF27
:10174C008D1700000000AD0BD843000001460C23A0
:10175C0009484B4370B5C418D4E90E5600224033E7
:10176C00A263184402F0A9FA2DB132462B46034865
:10177C00BDE87040184770BD98010020C4410000BE
:10178C0010B1012804D07047034B1B6C5B0701D1CF
:10179C00FFF7DCBF704700BF9801002008B54FF081
:1017AC002003EFF3118183F31288BFF36F8F124A7A
:1017BC00136843F0020013F0010310600CD04FF0DB
:1017CC008042D2F80C34D2F80C2413F0010303D06D
:1017DC000A4802F072FA012381F31188BFF36F8F6C
:1017EC0023B1BDE808400020FFF7B0BFBDE80840BA
:1017FC00012000F0EDBE00BFE8010020D801002060
:10180C0010B5074C23782BB94FF4A57002F0ACFC43
:10181C0001232370BDE81040002000F0D9BE00BFAA
:10182C0059030020094BBFF35B8F53E8002F22F0C4
:10183C00020143E800100028F7D1BFF35B8FD307F8
:10184C0002D4012000F010BF704700BFE801002057
:10185C001FB500220123CDE90223094ACDF800D09F
:10186C006B46CDF804D002F05EFA002805DB4FF48D
:10187C0080420023684601F0EDFD05B05DF804FBE5
:10188C00053D00002DE9F8433A49BFF35B8F06464E
:10189C00012251E8003F41E800200028F9D1BFF3B4
:1018AC005B8F33B9344935484B60CB608A6002F0AA
:1018BC00F1F8731E012B32D8012E07D14FF0804363
:1018CC00D3F81C3403F00303012B28D002F002FCE4
:1018DC00044618B92A4B1B78002B44D14FF0200337
:1018EC00EFF3118583F31288BFF36F8F0124254F1B
:1018FC00DFF89480DFF894904FF08042D2F81834DF
:10190C00D2F81824D2030CD503F00303012B01D019
:10191C00012E06D10CB385F31188BFF36F8FBDE890
:10192C00F883ACB12846FFF7E3FA4FF08042D2F8C7
:10193C001835002BE0D139680029DDD03B603B68BD
:10194C000123C2F81835C8F88031C9F80030D3E744
:10195C000021212001F0ECFCE7E74FF0804302224C
:10196C00C3F80423DBE74FF080430222C3F80823BB
:10197C000546BCE7EC01002088010020B4010020E2
:10198C006B0700200401004000E100E0080000406B
:10199C0008B5084B0848186002F0C7FA38B1074878
:1019AC00FFF716FE0548FFF77BFA002008BD6FF025
:1019BC001200FBE7F0010020DC410000CD19000013
:1019CC000A2838B5074D044604D1286883680D21D0
:1019DC005B68984728688368E1B25B689847204643
:1019EC0038BD00BFF001002008B5094B1A786AB960
:1019FC000121197006200521FFF700FB0620FFF7D7
:101A0C00DFFA044B4FF00042C3F80423002008BD5A
:101A1C005A0300200060004073B50D46416806690A
:101A2C00097A05F01F04B2F5A03F44EA41140CD129
:101A3C0004F01F014FF0A04001F5E07150F82110A7
:101A4C00C80707D56FF0850093E0B2F5005FF16829
:101A5C0000F09180F0680121A94001437069F160A8
:101A6C000121A940B2F5A03FB2690CBF08438843DD
:101A7C00B3F5C02F0CBF0A438A43B261326970615F
:101A8C00B3F5802F0CBF114322EA0101464A3161A4
:101A9C00D2F804330020DBB200F5A27152F8211009
:101AAC00C1F304218C426BD123FA00F1C90767D52D
:101ABC00830003F1804303F5C043D3F8101521F0E4
:101ACC000101C3F8101501238340C2F80833C0B2DA
:101ADC0000F044FE2046002102F040F9F068E84096
:101AEC0010F0010045D07069E84010F001024ED0B2
:101AFC00B369EB40DB075FBF316921FA05F505F0EF
:101B0C000105C5F102050DF1070054BFEDB2032527
:101B1C0000F046FE254B984236D19DF807108B00FD
:101B2C0003F1804303F5C0432402D3F8102522F4BB
:101B3C00473222F44072C3F81025D3F8102504F470
:101B4C00F85414438A0002F1804202F5C24244EA7E
:101B5C0005450020C3F8105510601268D3F8102505
:101B6C0042F00102C3F810250F4A01238B40C2F842
:101B7C00043302B070BD0120A84021EA00016DE7DA
:101B8C000130082888D1A5E76FF01200F1E7316920
:101B9C00E94001F00101C1F103012046C9B202F094
:101BAC00DDF81046E5E700BF006000400000AD0B1B
:101BBC002A4B70B546682A48134083423ED00DD854
:101BCC00062B15D005D89BB1022B39D06FF0150020
:101BDC0033E0B3F5801FF9D1012309E0214883429A
:101BEC0030D0B3F5A00F2FD0B3F5800FEED1022378
:101BFC00D00654BFC2F34015032582F4807412F44E
:101C0C00007FC2F34020C4F3002407D012F4006F0D
:101C1C0076681BD001228A40C6F8082540EA4402A7
:101C2C0001F01F0142EA032301F5E0714FF0A042DD
:101C3C0043EA850342F82130002070BD0723D7E723
:101C4C000423D5E70523D3E70323D1E7520542BF8D
:101C5C0001228A40C6F80C25E0E700BF0600F00020
:101C6C000600100002004000464A2DE9F0471668B5
:101C7C00002E5AD0444BD3E90514D8681B69214374
:101C8C0020EA01084FF0A0414546D1F810455C40D0
:101C9C0028EA040401274FF0000A89467DBB156031
:101CAC0013683A48002301251F46D0F8042305FA8F
:101CBC0003F1114211D09A0002F1804202F5C242A6
:101CCC00116851B103F5A27150F821101760C1F3DE
:101CDC00042105FA01F112680C430133082BE4D1FD
:101CEC002CBB56B1284CD4E90510E268014322EA1A
:101CFC00010201250026002A31D1BDE8F0872F42D0
:101D0C000FD017EA080F0AF01F0008BF00F5E073A8
:101D1C004FF0000108BF59F8233002F01FF825EAF4
:101D2C0007050AF1010A7F00B8E73446B9E7164BFC
:101D3C0059680029D5D00D68154F002D38BF0025E6
:101D4C008A68224002D04B6838469847002DC8D08C
:101D5C002B68002B38BF002329461D46F0E715429F
:101D6C000CD02169F14001F00101C1F10301C9B2AC
:101D7C0006F01F0001F0F2FF22EA050201366D00A9
:101D8C00B9E700BF7C610040F40100200060004016
:101D9C000C42000070B54B79012B24D18B79032BAD
:101DAC0021D1CA792AB1012A1DD143685B689B07EE
:101DBC0019D00C7914B1022C15D10E240B6845687E
:101DCC00B3F5164F2D6862D02BD8B3F5165F61D0E2
:101DDC0014D8B3F5966F5FD008D8B3F5967F5ED064
:101DEC00B3F5167F5ED06FF085004FE0B3F5166F3C
:101DFC005BD0B3F5965FF6D1364B3CE0B3F5E14FD3
:101E0C0056D007D8B3F5615F54D0B3F5964FEAD1ED
:101E1C00314B30E047F61226B342E4D14FF40003C5
:101E2C0029E0B3F5613F47D013D8B3F5963F46D0C0
:101E3C0009D84DF6C026B34243D0B3F5614FD2D189
:101E4C004FF46B0317E0B3F5E13FCCD14FF0EB73DC
:101E5C0011E0B3F5612F37D008D8204EB34236D0FD
:101E6C00B3F5E12FBFD14FF0E86304E01C4EB34251
:101E7C00B9D14FF08053C5F82435036903C9224307
:101E8C000433C5F86C2583E80300002070BD4FF4C3
:101E9C001D03F0E7134BEEE74FF49E23EBE74FF4F3
:101EAC00A033E8E74FF41C33E5E74FF41D23E2E7DA
:101EBC000D4BE0E70D4BDEE74FF06C73DBE70C4BA3
:101ECC00D9E74FF46503D6E74FF07063D3E74FF0D3
:101EDC008063D0E700B0130000A04E0090D0030048
:101EEC0040420F000050270000C0750000F03A007F
:101EFC0000903A01F8B5066905460F4602F0EAF87B
:101F0C0010B92C4B1B7883B94FF02003EFF31184DD
:101F1C0083F31288BFF36F8F284601F0C8FF28BBEC
:101F2C0084F31188BFF36F8FEEE76424284601F029
:101F3C00BEFF70B9012001F0EEFF013CF6D100218B
:101F4C00212001F0F5F9F0E784F31188BFF36F8FCE
:101F5C00F5E74FF02003EFF3118483F31288BFF3FE
:101F6C006F8F284601F0A3FF0028EDD006F8107FF4
:101F7C0069680B680122C3F84465C3F84825002240
:101F8C00C3F82021D3F82001C3F85821D3F85821E5
:101F9C004A68D20641BF0822C3F800254FF48002DC
:101FAC00C3F8042301229A6084F31188BFF36F8F66
:101FBC00F8BD00BF6B070020F8B5002207460121D1
:101FCC000220FFF71BF80220FEF7FAFF7D683E693E
:101FDC002C68D5F808C00023C4F800354FF0A04198
:101FEC000CF01F0301229A4003F5E0733760C1F82F
:101FFC000825032241F82320EA68501C07D0287ECC
:10200C0002F01F0303F5E073800041F82300C4F8CD
:10201C000CC5C4F814252A69531C09D0697E02F03A
:10202C001F0303F5E0734FF0A040890040F8231024
:10203C006969481C0CD001F01F034FF0A04C012023
:10204C00984003F5E073CCF8080503204CF8230006
:10205C00C4F808153969C4F8102538460431FFF75F
:10206C0099FE0746002845D16B68190719D506F16A
:10207C00120000F0CDFB224B98423DD1B07CC30046
:10208C0003F1804303F5F83304F10C0204F590716D
:10209C00C3F81015C3F814251A4A01238340C2F85B
:1020AC0004350823C4F80035EB6801330CD0002349
:1020BC00C4F81031D4F8103106F11103C4F83435DA
:1020CC000123C4F8383523606B681A075CBF4FF4E2
:1020DC008072C4F80423DB0644BF4FF48003C4F8B9
:1020EC00043310360023C4F84465C4F84835012382
:1020FC00A360E3603846F8BD6FF00407FAE700BF51
:10210C000000AD0B00F00140194970B5044622F0F7
:10211C007F460868C1E90023A6F50013101AB3F531
:10212C00400F4FF000050AD2124B19680A060B0A31
:10213C009219114943F10003C1E90023012501F073
:10214C001BFBA30003F1804303F58833D3F8402530
:10215C00B2420BD11DB94FF40002C3F84025074B16
:10216C004FF4803000FA04F4C3F8444370BD00BF50
:10217C0058000020180200204000002000100140F0
:10218C0010B501238340114ABFF35B8FDC4352E847
:10219C00001F01EA040C42E800CEBEF1000FF6D19C
:1021AC00BFF35B8F4FF4803202FA00F002F18042F1
:1021BC0002F58052C2F80803BFF35F8FBFF36F8F35
:1021CC000B4214BF0120002010BD00BF14020020E0
:1021DC000123124ABFF35B8F834052E8001F19435F
:1021EC0042E8001CBCF1000FF7D1BFF35B8F0C4A27
:1021FC004FF480338340C2F804330A4BBFF35B8F38
:10220C001B68BFF35B8F23FA00F0C30742BF064B7A
:10221C004FF40032C3F80021704700BF14020020B5
:10222C00001001401002002000E100E00D4B1B6883
:10223C00190A1806BFF35F8F0B4BD3F80435C0187F
:10224C0041F10001B3F5801F0AD2084BD3E90023FA
:10225C00994208BF904203D210F1807041F1000105
:10226C00704700BF18020020001001404000002001
:10227C002DE9F04F85B016461F460546FFF780FF47
:10228C000190FFF7D3FFB94208BFB0427FD2B6EB43
:10229C00000867EB010900234FF080724B4508BF23
:1022AC004245C0F08580444B03EB0513D3E9022370
:1022BC009F4208BF964254D04FEA85094FF4803BA9
:1022CC0009F1804905F150080BFA05F209F5883936
:1022DC004FEA88081FFA88F80292384AD9F8400564
:1022EC0026F07F4308F1804808F588381C46934651
:1022FC00D2F804A5A0EB0A0020F07F402AF07F4121
:10230C000128C9F8401505D10393132001F02CFFC7
:10231C002A4A039B02990AF1020CA4EB0C0020F050
:10232C007F40B0F5000F88BF64460020C8F800005D
:10233C00D8F80000CBF8441324F07F40C9F84005CE
:10234C00DBF80405824506D0201A023820F07F40C5
:10235C00B0F5000F19D8E41A24F07F44321947F174
:10236C000003154C290104EB0510C0E902230E9A59
:10237C000F9B625043600024019B13B12846FFF76A
:10238C0027FF204605B0BDE8F08F2046B0E70123BB
:10239C000B4ABFF35B8FAB4052E8001F194342E876
:1023AC0000100028F8D1BFF35B8F32463B46D8E7CC
:1023BC006FF01504E0E700BF48000020001001405A
:1023CC00100200202DE9F743344CD4F804339A075B
:1023DC0009D5334B1A6832B100221A60314A1B6896
:1023EC001368013313604FF02003EFF3118283F372
:1023FC001288BFF36F8FD4F80433DB0312D5BFF30D
:10240C005B8F294B53E8001F21F0010043E80006C5
:10241C00002EF7D1BFF35B8F244B002936D11968FE
:10242C00002933D1002382F31188BFF36F8F53B38C
:10243C00FFF7FCFE06464FF02003EFF3118083F309
:10244C001288BFF36F8F1A4BD3E90289494508BF35
:10245C0046454FF000021ED34FF0FF364FF0FF37CA
:10246C00D3E90015C3E902671A604FF48033C4F84E
:10247C00483380F31188BFF36F8F21B1009542462A
:10248C004B460020884703B0BDE8F083002119605B
:10249C001B680123C7E71146EBE700BF00100140A2
:1024AC0004110140180200201002002040110140CC
:1024BC004800002073B51A4B1A4D00244FF0FF3022
:1024CC004FF0FF31C5F80845C3E902014FF48033E2
:1024DC00C5F80433144B02264FF400320121C5F821
:1024EC0004631120C3F880212246FEF787FD1120DA
:1024FC00FEF766FD0D4AC5F80463012313600C4A10
:10250C002B6013600B4B0C4A009301940023204664
:10251C00FFF7AEFE3046FFF7B5F9204602B070BDAE
:10252C00480000200010014000E100E008100140CC
:10253C001402002015210000FFFF7F00144B13B57F
:10254C00B0F1FF3F08BF1846441E002C1EDD9C4214
:10255C00A8BF1C46FFF76AFE0E4B0F49D3E90023B8
:10256C00801AB0F5000F28BF00240130044408483D
:10257C000091844228BF044612194FF000000190CC
:10258C0043F10003FFF774FE02B010BD0024E1E735
:10259C00FFFF7F00580000201521000008B5FFF751
:1025AC0045FE024B1B68C01A08BD00BF5800002036
:1025BC00044B1A7922B9012218609A80024870479C
:1025CC00024870471C0200200000AD0B0C00AD0B44
:1025DC0030B510B1012833D030BD4FF08043D3F863
:1025EC001824D3F8181411F4803F194624D002F0A3
:1025FC000302012A20D1C3F81825164B00221A60B9
:10260C001B684FF080430222C3F80423124AD0689F
:10261C0040F08073D360114B1C6844F001011960C9
:10262C005D685968491BB1F50A5FFAD31C600C4B05
:10263C00D06001221A60CFE70023C1F81835DCE71F
:10264C00084B00221A601B684FF08043C3F8040348
:10265C001860C1E704010040F0ED00E0001000E05C
:10266C00080000400001004038B510B1012818D016
:10267C0038BD4FF080430222C3F80823184A10607B
:10268C001268184A0121116042F210751C46D4F8E8
:10269C001834DB03ECD5012001F03DFC013DF6D1F3
:1026AC00E6E7114B4FF080440022C4F808031A608F
:1026BC001B680E4B42F210751860D4F80C34D4F829
:1026CC000C24D20303F0010305D523B1012001F042
:1026DC0022FC013DF1D1064B00225A71C8E700BF24
:1026EC00040100400C0000400001004004000040C8
:1026FC001C020020164B1A6810B56AB100221A6031
:10270C001B684FF080430122C3F80823114B587902
:10271C0010B95A711B6898470F4B1A6872B1002296
:10272C001A601B684FF08043D3F81824D3F81814A0
:10273C00920704D10122C3F818259A6010BD022219
:10274C00C3F80823034BBDE810401B680120184751
:10275C00000100401C02002004010040012303FA88
:10276C0000F010F0FF0F12D04FF02003EFF31181A7
:10277C0083F31288BFF36F8F064AD36C23EA0000F1
:10278C00D06481F31188BFF36F8F034870470348FF
:10279C00704700BF240200200000AD0B0400AD0BFD
:1027AC002DE9F0410546DFF860E01648DFF85C8063
:1027BC000024FF220126E3B24FF02001EFF3118C2D
:1027CC0081F31288BFF36F8F22FA03F1C9070AD580
:1027DC00DEF84C1006FA03F7394201BF3943CEF844
:1027EC004C1040462B708CF31188BFF36F8F404513
:1027FC0005D006FA03F39A4304F10104DBD1BDE8DA
:10280C00F08100BF0200AD0B240200200000AD0BD4
:10281C002DE9F041144A154E154F05461548002474
:10282C004FF0010E5FFA84FC4FF02003EFF3118898
:10283C0083F31288BFF36F8F0EFA0CF3134207D099
:10284C0031680B4201BF1943316085F800C038462E
:10285C0088F31188BFF36F8FB84203D09A4304F109
:10286C000104DFD1BDE8F081FFFF0F0074020020EE
:10287C000000AD0B0200AD0B044B1868421C04BFEA
:10288C00034B1878831F5842584170473001001091
:10289C00E00F00F0074B1B78062B09D1064B1B6889
:1028AC00C3F30313033B042B02D8044AD05C7047D8
:1028BC0000207047E00F00F0E80F00F09E4400008D
:1028CC00024AD2F80034002BFBD0704700E00140E4
:1028DC0010B5FFF7D1FF28B1814B824A1B68C3F3B7
:1028EC0004231360FFF7D6FF10B17F4B7F4A1A60A9
:1028FC00FFF7C2FF28B17E4B7E4A1B68C3F34233FD
:10290C001360FFF7C7FF20B17B4AD36823F08073B5
:10291C00D360FFF7B1FF40B14FF080430022C3F802
:10292C000C21C3F81021C3F83825FFF7B3FF10B101
:10293C00724B03221A60FFF7ADFF40B1704B0522BA
:10294C001A6001229A6700229A603F225A606D4BEE
:10295C001A68511C0BBF6C4B6C4B1A781B6802BF6E
:10296C0008331B68C3F30313062A4DD1033B042B16
:10297C0003D8674AD35C002B46D04FF08052654B8E
:10298C00D2F80414C3F82015D2F80814C3F824158F
:10299C00D2F80C14C3F82815D2F81014C3F82C155F
:1029AC00D2F81414C3F83015D2F81814C3F834152F
:1029BC00D2F81C14C3F84015D2F82014C3F84415EF
:1029CC00D2F82414C3F84815D2F82814C3F84C15BF
:1029DC00D2F82C14C3F85015D2F83014C3F854158F
:1029EC00D2F83414C3F86015D2F83814C3F864154F
:1029FC00D2F83C14C3F86815D2F84014C3F86C151F
:102A0C00D2F84424C3F87025FFF736FF28B1424BA7
:102A1C00424A1B6803F04F031360FFF72DFF48B1C8
:102A2C004FF08043D3F80024D20744BF6FF001026B
:102A3C00C3F80024334B1B68062B20D1334B1B6887
:102A4C00033B042B02D8364AD35C43B1354A136896
:102A5C0043F4806313602B4B1B68062B0FD12B4B5D
:102A6C001B68033B042B02D82F4AD35C3BB14FF0BD
:102A7C001023D3F808224FF08043C3F858254FF0A9
:102A8C001023D3F80022002A03DBD3F80432002BE6
:102A9C0022DA26490123C1F80435FFF711FF4FF064
:102AAC0010201524C0F80042FFF70AFFC0F80442BA
:102ABC00FFF706FF0023C1F80435FFF701FFBFF352
:102ACC004F8F1B491B4BCA6802F4E0621343CB6067
:102ADC00BFF34F8F00BFFDE7174B184A1A6010BDAC
:102AEC00240300104035014074C007400DF0ADBA0E
:102AFC00440200103C050040F0ED00E0A005004051
:102B0C001056004030010010E00F00F034010010AE
:102B1C008F44000000C0004058020010E40E00403A
:102B2C00944400003C1700409944000000E0014030
:102B3C0000ED00E00400FA05200000200090D00316
:102B4C0010B5144C144A1549032323616361144BCB
:102B5C00A261E3614FF4806323620023A36263628A
:102B6C00E36222660F4A6266E01D1022A2662367AA
:102B7C00E366636701F009F8BFF35F8F0A492046EB
:102B8C0001F003F8BFF35F8F2023A371BFF35F8FB6
:102B9C0010BD00BF78020020A3440000AC4400002C
:102BAC006B0300205B030020B04400000E4B70B59B
:102BBC0053F82040013053F82060A64200D870BD75
:102BCC00D4E900352846984765B1EB6830B1002848
:102BDC00B8BF4042FF28A8BFFF2018705A7842F0B7
:102BEC0001025A700834E8E74444000070B5054609
:102BFC0010B90024204670BD0378002BF9D00F4A81
:102C0C000F4C1646944208D10D4CB442F1D02046DC
:102C1C0001F08BF950B91834F7E7204601F085F92B
:102C2C0010B12368AB42E5D01834EBE72168284695
:102C3C0000F0C5FF0028EED1DCE700BF2442000005
:102C4C00C441000008B5094C4FF02002EFF311838A
:102C5C0082F31288BFF36F8F01F058FAA061FEF770
:102C6C00D3F80028F0D1FEF735F9EDE7200300206A
:102C7C0030B5002387B00122CDE904230F22CDE922
:102C8C0002320D4C0D4A01930D49182304EBC0146C
:102C9C0003FB00234FF4B075009305FB0011094BA7
:102CAC004FF4A072204600F0FFFB637B23F004037B
:102CBC00637307B030BD00BF60000020200300200C
:102CCC00A00B0020512C000008B50A4B0122022059
:102CDC001A70FFF76BFF00F0EFFD0320FFF766FFA4
:102CEC0000F014FCFDF76EFB034A137B23F0010389
:102CFC00137308BD6B070020E00000200248034A54
:102D0C000021121A00F072BF400000206C07002056
:102D1C0080B5DFF8D880A6B088F308882D4D2E4EEC
:102D2C006B69DFF8CC9043F4007300246B61E023F3
:102D3C0085F82230EC772C766C76AC7685F82040D2
:102D4C006B6A43F4E0236B6285F82340FEF71CFBAF
:102D5C00FEF7BAF84FF0FF33AB62EB62FEF70AFCFA
:102D6C00FEF77AFB40F20113ADF8243006ABB360EA
:102D7C00CDE91F4401F0D8F82046FFF717FF0120DA
:102D8C00164DFFF713FF00F039FA154B059301238D
:102D9C0014490094CDE903434FF480624B46CDE9CE
:102DAC0001442846F56100F07FFB6A7B22F00402A7
:102DBC006A730746284601F016F92046FFF758FFBC
:102DCC00094BF3604A46394628463475C6F80480E8
:102DDC00FEF798F900ED00E020030020E000002051
:102DEC00B744000080070020600000202015002060
:102DFC00D52C000010B5084C23685BB1FFF7CEFB57
:102E0C0003462068054A0344BDE8104013610021C5
:102E1C0001F08CB910BD00BF50030020200300202E
:102E2C00F8B504460D464FF02003EFF3118683F3FB
:102E3C001288BFF36F8F104B00224FF4004740F203
:102E4C00E73000211A61E7FB040100234FF47A728A
:102E5C00FDF73EF9002C094B09DC1860084B1D608E
:102E6C00FFF7C8FF86F31188BFF36F8FF8BD0228F8
:102E7C00B8BF0220F1E700BF200300205003002060
:102E8C004C03002049B9EFF3058030B9054BDA69E2
:102E9C009B689A4201D0FEF7E5B881F31188BFF325
:102EAC006F8F7047200300204FF02003EFF3118148
:102EBC0083F31288BFF36F8F044B9A68D37B013B6B
:102ECC00D37381F31188BFF36F8F704720030020F9
:102EDC0038B502460C480D4D01F07BF8044600B99C
:102EEC00EC68AB684AB95A7BD20606D1A26922B902
:102EFC00DA897F2A01D9EB6138BD9C4201D0FFF7FA
:102F0C0079FFEC61F8E700BF4003002020030020AC
:102F1C0070B590F90D20437B002A014604DA03F0CA
:102F2C007F03437301F02DF84B7B174A63F07F034B
:102F3C0010464B7350F8203F556A834208BF00235C
:102F4C00002B38BF0023CBB191F90E6093F90E40E2
:102F5C00A6420FD0A41B002C0CDD5868C1E9003030
:102F6C00016059609068431A5842BDE8704058415E
:102F7C00FFF7AEBFAB4201D01B68E4E7C1E9000527
:102F8C0029605162EEE700BF2003002070B50146B6
:102F9C004FF02003EFF3118483F31288BFF36F8F8C
:102FAC00164B174A98681568A8421D4606D1FFF7BC
:102FBC0021FF84F31188BFF36F8F70BD002616605C
:102FCC00104A1268BAB1C2897F2A14D8427BD20641
:102FDC0011D10D4A90F90E60126896420BDB0B4A28
:102FEC00904208D01A698A4202DCFFF791FFDEE7B3
:102FFC00521A1A61DDE700232B61DAE72003002067
:10300C0048030020500300204C03002060000020E7
:10301C0070B490F90D30427B002B2DDBD3062BD1F5
:10302C0083694BBB154962F07F0242730A464D6AB5
:10303C0052F8204F944218BF2346002B38BF002370
:10304C00ABB190F90E6093F90E40A6420BD0A41BC5
:10305C00002C08DD5A68C0E900321060586070BC62
:10306C000020FFF735BFAB4201D01B68E8E7C0E991
:10307C00002528604862F2E770BC704720030020EE
:10308C0010B54FF02002EFF3118482F31288BFF3D6
:10309C006F8F427B510704D484F31188BFF36F8F79
:1030AC0010BD22F004024273FFF7B2FF2146024822
:1030BC00BDE81040FFF7E6BE6C07002008B590F99C
:1030CC000D20437B002A014604DA03F07F0343738F
:1030DC0000F057FF044B9868431A58425841BDE81A
:1030EC000840FFF7F5BE00BF200300202DE9F0419A
:1030FC00064614461D464FF02003EFF3118783F369
:10310C001288BFF36F8F00F0A0FF87F31188BFF315
:10311C006F8F6B1C08BFB4F1FF3F08D022462B46C3
:10312C0006F118000349BDE8F04100F09DBABDE876
:10313C00F08100BF1340000010B5074B9868074B97
:10314C000C4618601146DDE90223FFF7CFFF20463D
:10315C00BDE81040FDF786BF200300204803002087
:10316C0070B50446183000F0BBFF4FF02003EFF3AE
:10317C00118683F31288BFF36F8F94F90D20637B54
:10318C00002A05DA03F07F036373204600F0F9FE92
:10319C000B4D637BA86843F010036373031B584209
:1031AC005841FFF795FE86F31188BFF36F8FAB681C
:1031BC00A34203D1BDE8704000F001BF70BD00BF59
:1031CC002003002010B54FF02003EFF3118483F39C
:1031DC001288BFF36F8F084B9A68D37B0133D3737C
:1031EC000020FFF775FE84F31188BFF36F8FBDE8E5
:1031FC00104000F0E4BE00BF20030020044B00216F
:10320C0003F12002C3E908220846FFF709BE00BFFC
:10321C0020030020F8B54FF02003EFF3118483F363
:10322C001288BFF36F8F1B498868437B03F07F03C1
:10323C00437300F0A6FE8A68537B084663F07F0355
:10324C00537350F8203F4E6A834208BF0023002B73
:10325C0038BF0023CBB192F90E7093F90E50AF42E8
:10326C000FD0ED1B002D0CDD5968C2E900310A604E
:10327C005A600120FFF72CFE2046BDE8F840FDF710
:10328C00F1BEB34201D01B68E4E7C2E9000632602C
:10329C004A62EEE7200300202DE9F04104460D467A
:1032AC0054EA050104D1FFF7B5FF0020BDE8F08119
:1032BC006FF001010A1A4FF0FF3161EB0503012A8F
:1032CC0073F100032ADA00F04BFF06194FF02003CC
:1032DC00EFF3118883F31288BFF36F8F114F124BEA
:1032EC00B8681860FFF7EAFEB868104922462B460A
:1032FC00183000F0B9F9BA68537B43F010035373DC
:10330C004046FDF7AFFE00F02BFF301A66EB0601CE
:10331C00012871F10003B8BF0020C7E76FF0010668
:10332C00361AD3E720030020480300201340000086
:10333C0008B50B46013308BFB0F1FF3F06D1084B6F
:10334C009868FFF70DFF4FF0FF3008BDFFF7A4FFA3
:10335C004FF47A7380FB0323D00B40EA4340F4E72D
:10336C0020030020014B9868704700BF2003002009
:10337C002DE9F04104464FF02003EFF3118683F35F
:10338C001288BFF36F8F437B1A0705D586F311881C
:10339C00BFF36F8FBDE8F08123F0200242F00801EB
:1033AC00D20920D14173A36813B1204600F0F1FD7E
:1033BC0004F1180000F094FE04F158074FF00008D7
:1033CC00A56DBD4200D0B5B90120FFF781FD104BB2
:1033DC009B68A342DAD1EFF30583002BD6D130469C
:1033EC00FDF740FED2E703F05F0343F0080343739D
:1033FC0000F0C7FDD7E7284600F0CBFD05F118001B
:10340C0000F06EFEC5F878802846FFF701FED7E77E
:10341C002003002038B504464FF02003EFF311854C
:10342C0083F31288BFF36F8F00F03CFE48B100228B
:10343C00826700F0D8FD29460548BDE83840FFF703
:10344C0021BDD4E902329A4218BF0133A360F2E7DE
:10345C006C07002037B514461D464FF02003EFF3E0
:10346C00118183F31288BFF36F8F836843B1013BE3
:10347C00836081F31188BFF36F8F002003B030BDE0
:10348C0054EA050306D181F31188BFF36F8F6FF0F7
:10349C000F00F3E70246CDE900450248FFF74CFE6A
:1034AC00ECE700BF6C0700202DE9FF410E9E067370
:1034BC00042646730D9E867300F158050F46D61DE3
:1034CC00C0E916550C9A002526F007062037C0E9EE
:1034DC000655C0E919768560C573C56606F12008E6
:1034EC0002920B9A019288440A9A00924246044630
:1034FC00FDF7D2FD044B65659B6803B11B6F236719
:10350C00404604B0BDE8F081200300202DE9F047CF
:10351C002A4E2B4D86B0B046B54205F1300410D37F
:10352C00FFF7C2FC264CDFF89CA04FF4004940F298
:10353C00E7360027444521D306B0BDE8F047FFF736
:10354C0041BE54F8043C059354F8103C049354F8D1
:10355C00143C039354F8183C029354F81C3C01930C
:10356C0054F8203C009354E90A2354E90C01FFF76A
:10357C009BFF54F8303C5D652546CDE7636A5A1CC9
:10358C000DD023EAE37330463946C9FB0301B94237
:10359C0008BFB042256804D12846FFF771FD3034CE
:1035AC00C8E74FF47A720023FCF792FD02460B46F3
:1035BC0005F11800514600F057F8F0E73C000020E8
:1035CC003C00002013400000034B1B680BB9FEF7B6
:1035DC00E5BF0020704700BF5403002030B50368DE
:1035EC0068B10A4A5268904209D043B1D3E9042128
:1035FC00D0E90445121945EB0101C3E904214268E5
:10360C0013605A600023C0E9003330BD2400002051
:10361C0038B5134B1C689C4208BF0024FFF7D4FF3D
:10362C000546BCB1D4E90401401B61EBE5710128EE
:10363C0071F1000311DB6FF000420023824273EB47
:10364C00010400DA1046074B1B6913B19842A8BF5E
:10365C00184638BD6FF00040F5E70020F3E700BFD7
:10366C002400002020030020B3F1FF3F08BFB2F17B
:10367C00FF3F2DE9F74F044692469B4673D081607D
:10368C004FF02003EFF3118583F31288BFF36F8F94
:10369C006FF00103B3EB0A084FF0FF3262EB0B093A
:1036AC00B8F1000F79F100011CDB3048D0E90010B3
:1036BC005B1A62EB0002B3EB0A0662EB0B07012EFE
:1036CC0077F10003BCBF01260027C4E90467284A30
:1036DC00D2E9003C93421ED1C4E9002CCCF8004046
:1036EC0054602DE0FFF770FF1AF1010300934BF1CA
:1036FC0000030193DDE90023121843EBE073C4E9E6
:10370C000423E4E7B6EB080067EB09016345C4E961
:10371C000401E1D01B68002BDED0D3E90489D4E985
:10372C000467464577EB0901ECDAB8EB060069EB68
:10373C000701C3E904015968C4E900310C605C60FD
:10374C00136893420BD09C4209D1FFF761FF18B16B
:10375C00084B1B69834202D00021FEF7EFFE85F374
:10376C001188BFF36F8F03B0BDE8F08F60010020AC
:10377C0024000020200300202DE9F74F0646FFF718
:10378C0005FC4FF02003EFF3118483F31288BFF391
:10379C006F8F2C4DDFF8B0A0DFF8B0B02E60514623
:1037AC00D5F800C0DBF800006246D3175845DAE9BB
:1037BC000089CDE900230DD060B1D0E90467B44590
:1037CC00BB411EDA009BB6EB030C019B67EB0306B7
:1037DC00C0E904C6009B13EB0802019B4FF00006E6
:1037EC0043EB0903C1E900232E60FFF711FF3146BB
:1037FC00FEF7A4FE84F31188BFF36F8F03B0BDE80E
:10380C00F08F18EB06084FF000024FF0000349EB65
:10381C00E679C0E90423ACEB0606CAE900892E6000
:10382C00FFF7DCFE84F31188BFF36F8F8368984732
:10383C004FF02003EFF3118483F31288BFF36F8FE3
:10384C000149ADE754030020600100202400002052
:10385C0010B54FF02003EFF3118483F31288BFF3FC
:10386C006F8FFEF79BFE064BD3E90023121843F132
:10387C00000384F31188BFF36F8F1046194610BDF7
:10388C006001002008B50648064A0749121A00F0E4
:10389C00A2F9BDE80840054A0549064800F09BB965
:1038AC00000000203C000020F0440000000000005C
:1038BC00F044000000000020024A0349034800F0D5
:1038CC0039B900BFEE440000BC440000C8440000FD
:1038DC002DE9F74F9946D37814466F2BA3F141028B
:1038EC0006460F4601922DD028D8582B14BF0A2516
:1038FC001025DDF83080AA464FF0000B52465B468F
:10390C0030463946FCF7E4FB092AD3B21FD83033D2
:10391C005F45DBB208BF564508F8013D01D3C845E9
:10392C0012D823789B0605D5082D16D1A37843F021
:10393C000803A370404603B0BDE8F08F03F0F70313
:10394C00702BD3E70825D4E706460F46D6E7019A35
:10395C00192A94BF37335733DAE7102DEAD1A378FD
:10396C0043F01003E5E72DE9F0410746884615467C
:10397C001E461446B442A4EB050002D33EB923788C
:10398C002BB114F8010B4146B8470028F2DABDE818
:10399C00F0817047034658B1426802F00302012AD5
:1039AC0003D0032A04D1026812B10020986070473A
:1039BC006FF0150070474268816002F00302032A21
:1039CC004FF0000203460CBF006810465A60704767
:1039DC00038B13F0070305D10368002B0CBF0020E9
:1039EC0003207047022B05D1438B002B14BF002002
:1039FC0004207047012B05D10368002B0CBF00205D
:103A0C0005207047002070472DE9F0410D46074610
:103A1C001946281D90461E46FFF7CDFF044638B1C7
:103A2C003346424629463846A446BDE8F041604735
:103A3C00BDE8F08110B44FF02004EFF3118284F351
:103A4C001288BFF36F8F416110BC0121FDF7AAB83A
:103A5C0010B50C4640B139B1081DFFF79BFF28B9D2
:103A6C00A36833F0030301D06FF0150010BD38B517
:103A7C000C46054658B151B10B6843B14B6833B194
:103A8C001C22002100F0B2F82C61002038BD6FF030
:103A9C001500FBE770B504460E46FFF7D9FF051E6F
:103AAC0031DB4FF02003EFF3118183F31288BFF366
:103ABC006F8F638B208B4FF6FF75AB4200F00702C4
:103ACC002ED0022A0ED1013363831546012381F3D4
:103ADC001188BFF36F8FB3B1002331462046FFF737
:103AEC0093FF10E0830701D0062A0ED10023336028
:103AFC00636893B9C4E90066154662B90A46204664
:103B0C000221FDF74FF8284670BD052A0CBF6FF057
:103B1C0085056FF004050023D9E71E606660EBE7AE
:103B2C006FF00A05F7E70022C0E9002282607047B7
:103B3C00002070470FB407B504A951F8040B01918C
:103B4C00FDF7B4F903B05DF804EB04B0704704461C
:103B5C0008B5084611461A46A047FFF703FCFDF7C7
:103B6C0069FC00F0ECB90146006800F0E8B90021EE
:103B7C000120FFF7F6BF08B5FDF7E4F9BDE80840F2
:103B8C00FDF7D6BA4FF0FF3070470139034611F8F4
:103B9C00012F0AB91A70704703F8012BF7E7034697
:103BAC0000201A5C02B970470130FAE70346002086
:103BBC001A5C0AB1884200D170470130F8E7431E05
:103BCC00013913F8012F11F8010F824201D1002A9B
:103BDC00F7D1101A704710B5431E0A44914200D118
:103BEC0010BD11F8014B03F8014FF7E7C9B20244BD
:103BFC000346934200D1704703F8011BF9E784B0E8
:103C0C0004AB03E907009DF80430062B08D14FF0F4
:103C1C0080430122C3F80025BFF34F8F20BFFDE77F
:103C2C0004B0704784B004AB03E90700002383F3AE
:103C3C001188BFF36F8F04B070470269CBB20C21AF
:103C4C0003FB0121086C00F0070070474FF02003C4
:103C5C00EFF3118283F31288BFF36F8F036813F0B5
:103C6C00C00301D08B4207D101230360002082F3F3
:103C7C001188BFF36F8F70474FF0FF30F7E710B527
:103C8C004FF02003EFF3118283F31288BFF36F8F91
:103C9C00036803F00704012C06D10160002082F3B5
:103CAC001188BFF36F8F10BD03F0C0038B4214BF9C
:103CBC004FF0FF306FF07700F1E74FF02003EFF398
:103CCC00118283F31288BFF36F8F036803F0C00374
:103CDC0043F00203036082F31188BFF36F8F7047C8
:103CEC00006910B4CBB21C2403FB0400002110BCEF
:103CFC0010470020FEF7B8BC1046FFF78BBB38B559
:103D0C00CCB20C2305466343006940338021184430
:103D1C00FFF79CFF002805DB696801EBC4046368AE
:103D2C009847002038BD2DE9F843CDB20C27046923
:103D3C006F43064607F14000802120449046994687
:103D4C00FFF79DFF002807DB3C44C4E90E8973682C
:103D5C0053F8353098470020BDE8F88300F01F0079
:103D6C00800000F1A040D0F8003723F4403343EA40
:103D7C000143C0F80037704743685B68D3F81035CF
:103D8C000B600020704743685B68D3F80405424021
:103D9C000A404240C3F804250020704743685B6822
:103DAC000020C3F80815704743685B680020C3F80F
:103DBC000C15704743685A68D2F804354B40C2F86A
:103DCC000435002070470369586830B558B1002499
:103DDC00814213D108685CB99C685860A14200D13B
:103DEC0098600020086072B9002030BD2846EFE7CB
:103DFC0020609868814208BF9C60F2E70568044621
:103E0C00002DF3D13AB15A680A60986859600028BD
:103E1C00EAD19960E9E76FF01500E6E743681B68A3
:103E2C00D3F80423D10518D5D3F82021AAB14FF02B
:103E3C002001EFF3118281F31288BFF36F8FD3F857
:103E4C00201131B10021C3F82011D3F82011012128
:103E5C00D96082F31188BFF36F8F42685268D20623
:103E6C0015D54FF02001EFF3118281F31288BFF3C7
:103E7C006F8FD3F8581111B10021C3F800154FF40E
:103E8C008001C3F8081382F31188BFF36F8F70475A
:103E9C0002690B46D2E9010183E803000020704758
:103EAC0043681B68D3F88004C3F8800470474268E9
:103EBC001368D3F8580140B95268120706D4D3F8E6
:103ECC002001003818BF012070470120704743685B
:103EDC0002691B68D3F8100148B1527C0A700020AB
:103EEC00C3F81001D3F8102101221A6070474FF06B
:103EFC00FF3070477047704708B50020FDF786FB10
:103F0C0008B50020FDF76CF818B9BDE80840FDF7BE
:103F1C0057B808BD004700F027B9FEF711BE08B529
:103F2C00FFF7FBFF002008BD704738B1C368188845
:103F3C00C0F30800A0F58073584258417047F8B59B
:103F4C0005460E464FF02003EFF3118783F31288DA
:103F5C00BFF36F8FFFF706FA314604462846FFF78A
:103F6C00CBFF87F31188BFF36F8F2046BDE8F84075
:103F7C00FDF760BA08B5FCF721FFBDE80840FFF774
:103F8C00BABFD0E9003213605A600023C0E9003395
:103F9C00704708B5FFF7F5FF437B23F0020343732B
:103FAC000023836008BD034620B9EFF305820AB9EC
:103FBC00FDF758B883F31188BFF36F8F70474FF03C
:103FCC002003EFF3118083F31288BFF36F8FFFF799
:103FDC00EABF03460068834203D0002838BF0020A4
:103FEC0070470020704710B54FF02003EFF3118499
:103FFC0083F31288BFF36F8FFFF70AF884F31188ED
:10400C00BFF36F8F10BD10B501464FF02003EFF3D7
:10401C00118483F31288BFF36F8F10F80B3C13F0ED
:10402C00280F0DD151F8103C18380BB1FFF7B1FF28
:10403C0011F80B3C23F0140301F80B3CFEF7E8FFDE
:10404C0084F31188BFF36F8F10BD38B504460D464D
:10405C00FFF734F8637B43F002036373B5B12B684D
:10406C00A5609D4208BF0023002B38BF00239BB1E5
:10407C0094F90E1093F90E20914208D0521A002A8E
:10408C0005DD5A68C4E9003214605C6038BD6A68AA
:10409C00934201D01B68EAE76B68C4E900531C60CB
:1040AC006C60F3E738B54FF02003EFF3118583F321
:1040BC001288BFF36F8FFFF78CFF044620B1FFF718
:1040CC0068FF183000F00CF885F31188BFF36F8F80
:1040DC00204638BDEFF30580003818BF012070472B
:1040EC0010B54FF02002EFF3118482F31288BFF366
:1040FC006F8F03683BB1FFF771FA002084F31188CE
:10410C00BFF36F8F10BD6FF01500F7E710B54FF0D0
:10411C002003EFF3118483F31288BFF36F8FFFF743
:10412C0077FA84F31188BFF36F8F10BD70B5044616
:10413C000D464FF02003EFF3118683F31288BFF383
:10414C006F8FFFF765FA012805DDA04203DB2946D6
:10415C002046FEF7F3F986F31188BFF36F8F70BD1D
:10416C0008B5FFF775FB08BD08B1FDF765BA7047D8
:08417C0070470000FEF7ACBB28
:0841840088BFFF7F010000006D
:10418C00E9150000000000002B3F000000000000BB
:10419C00F9160000C4410000C51F0000DC410000FE
:1041AC009D19000000000000C1240000F441000033
:0841BC00F51900000C4200009F
:1041C40078440000C8430000B44300002C000020E1
:1041D400980100206E4300007E4400002844000043
:1041E40014440000340000200C000020664300004A
:1041F400854400000000000000000000380000209A
:1042040000000000624300005C4400000844000019
:10421400E443000030000020F40100205C4300006F
:1042240001270000213F0000000000007B3B00004C
:10423400DC410000293E0000000000007B3B000040
:10424400000000007B3B0000000000007B3B0000FE
:1042540000000000751C0000000000007B3B000013
:10426400000000007B3B0000000000007B3B0000DE
:10427400000000007B3B0000000000007B3B0000CE
:10428400000000007B3B0000000000007B3B0000BE
:10429400000000007B3B0000000000007B3B0000AE
:1042A400000000007B3B000000000000D123000060
:1042B400000000007B3B0000000000007B3B00008E
:1042C400000000007B3B0000000000007B3B00007E
:1042D400000000007B3B0000000000007B3B00006E
:1042E400000000007B3B0000000000007B3B00005E
:1042F400000000007B3B0000000000007B3B00004E
:10430400000000007B3B0000000000007B3B00003D
:10431400000000007B3B0000000000007B3B00002D
:10432400000000007B3B0000000000007B3B00001D
:10433400000000007B3B0000000000007B3B00000D
:10434400000000007B3B0000000000007B3B0000FD
:08435400000000007B3B0000AB
:10435C00FF7FFF7FFF7FFF7FFF7FFF7FFF7FFF7F61
:0A436C00FF7FFF7FFF7FFF7FFF7FD1
:0A437600FFFFFFFFFFFFFFFFFFFF47
:104380000338FDD870470000000000200000000046
:1043900000000B06020000009C430000000000002B
:1043A000694400002400020700000020714400005E
:1043B0001E000B115D1800000B3D0000333D000096
:1043C00000000000473C0000A91700003118000061
:1043D0000D180000FF3C0000A11600005916000057
:1043E00000000000BD1B0000853D0000933D000063
:1043F000A93D0000B53D0000C13D0000251A0000A8
:10440000D33D000000000000FFFFFFFF0000005050
:1044100000000000DB3E0000011F0000AD3E000078
:10442000A11D00009D3E0000002000400B00000088
:104430000600000008000000070000000500000062
:10444000000000008C410000B4410000BC410000AD
:10445000C4410000C4410000F5FFFFFF4750494F31
:104460005F3000286E696C2900464C4153485F302C
:10447000005352414D5F3000434C4F434B00554178
:1044800052545F30007379735F636C6F636B00002D
:104490000001010100000001010000000001010015
:1044A0000000005465726D696E616C0052545400D6
:1044B000534547474552006D61696E0076322E378D
:1044C0002E302D6E637331002A2A2A20426F6F74BA
:1044D000696E67205A6570687972204F5320627543
:1044E000696C64202573202573202A2A2A0A00007B
:1044F000010000003D3B0000913B00000000000077
:1045000000C20100000103000000000000000000E4
:0C4510000090D0032400002024000020B4
:10451C00000000000000000000000000000000008F
:040000030000116D7B
:00000001FF
